:020000020000FC
:1000000070C11895C4C1189518951895189518952C
:10001000189518951895189563C3189518957A44EE
:1000200061746C675F5420302E316520302E31664C
:10003000203038303332332E323330370D0A0A0055
:100040000000623A20746573747320706F757220BB
:1000500064656275672C20433A636C656172206C3D
:1000600027454550524F4D2C20643A2073656172EC
:10007000636820312D776972652C20673A676F209D
:100080007265636F72642C20683A68656C702C200E
:10009000723A6C656374757265206465732076616D
:1000A0006C6575727320656E7265676973747265CD
:1000B00065732C20763A76657273696F6E0D0A004F
:1000C000C49AC498BC9AC39ABB9808950F931F937F
:1000D0003F930AE03095089410F4C49A01C0C49884
:1000E0001AD019D036950A95B9F73F911F910F9103
:1000F0000895B39BFECF0F931F9309E00CD00BD054
:100100000AD08894B39B08940A9511F04795F7CFCD
:100110001F910F91089515E81A95F1F70895EF933F
:10012000FF933F933591303021F43F91FF91EF9150
:100130000895CCDFF7CF0F931F932F9319D008D0DA
:10014000222311F430E3C2DF2F911F910F91089504
:10015000329503D0329501D008953F933F70230F1D
:10016000030F21F001E010E3310FB0DF3F9108955C
:1001700015D000E020E03F2DF0DF3E2DE9DF3D2DE2
:1001800008950F931F932F93F3DF3295E6DF3F938C
:100190003EE29CDF3F913295E0DFD2CF2F933F9339
:1001A000EF93FF9320E1FF24EE24DD24FF27000FCF
:1001B000111FDD1CEE1CFF1C2A9529F4FF91EF9105
:1001C0003F912F910895E0E132913D5F33FD3083FF
:1001D0003081305D37FD3083ED30B1F7E8CF692FE6
:1001E0006F706A3010F4606302C087E3680F792F84
:1001F00072957F707A3010F47063089587E3780FFA
:1002000008955527442760E13695279510F4400F4F
:10021000511F57954795379527956A95B9F70895D2
:10022000EE24FF1841E1001F111F4A9509F40895BB
:10023000EE1CFF1CE21AF30A20F4E20EF31E88946F
:10024000F2CF0894F0CF0F9304D00A95E9F70F91FD
:1002500008950F930AE004D00A95E9F70F910895E5
:100260000F9304E602D00F9108951F930F9314E1AA
:1002700007D01A95E9F70A95D1F70F911F910895C4
:100280000F930BE00A95F1F700000F91089500001D
:10029000000000000895B6E0BA95F1F7AA95D9F7E5
:1002A00008950F931F9303E016EFAFEFF4DF1A9555
:1002B000E1F70A95C9F71F910F910895E199FECFD3
:1002C0000F9300E00CBB0F913FBB2EBB0DBBE29A1E
:1002D000E19A0895E199FECF3FBB2EBBE09A0DB3A2
:1002E00008950FE511E00DBF1EBF00E806BD01E057
:1002F00006BD44D0E5DE3CE0E9DE19C038C03EE38F
:10030000E5DEF7DE423681F0433479F0443671F0B1
:10031000473669F0483639F1423751F0463739F1FE
:1003200037E0D4DE19D0EBCF31C212C241C093C145
:10033000EBC10F933F933DE0C9DE0FE430E2C6DE30
:100340000A95E1F73DE0C2DE3F910F9108953CE24E
:10035000BDDE30E2BBDE08953F933DE0B7DE3AE01C
:10036000B5DE3F910895E2E4F0E0D9DEC8CFEEE1DA
:10037000F0E0D5DEC4CF09E601BD0895A89500E000
:1003800004BF01B5086101BD00E001BD08954F93B0
:100390004FB74F9340916100442331F4ACDE40935A
:1003A000600041E0409361004F914FBF4F9118951D
:1003B00014C154612000C298C29ABA980895C29894
:1003C000BA9AA9E868DFC29ABA98ADE064DF07B3C9
:1003D00002FBAEEB60DF089508E0C298BA9A000015
:1003E0000000000000000000179510F4C29ABA98AF
:1003F000ADE051DFC29ABA98A1E04DDF0A9569F7E6
:10040000089508E01127C298BA9AA1E044DFC29A81
:10041000BA98A1E040DF1695B2991068ADE03BDFD5
:100420000A9589F708951F9308E011251795112D56
:1004300020F40F9308E110270F911795112E1F91AB
:1004400016951F930A9589F71F9108951CECC4DF38
:1004500014E4C2DFC29ABA9A24DFBA9808951EEB58
:10046000BBDF112428E0D0E0C4E6CBDF1993DBDF4B
:100470002A95D9F7C6DF199310926D000895DF937E
:10048000CF9301E006C0DF93CF9300916E00D0E0E0
:10049000CFE627E09991A3DE372F18DE362F16DE40
:1004A0003AE314DE2A95B1F7999199DE372F0EDEE3
:1004B000362F0CDE51DF0A9561F7CF91DF91089559
:1004C0007EDF15E589DF28E0199186DF2A95E1F7BF
:1004D000C6DF0895009164001091650025E030E0CA
:1004E00090DE022F132F28E030E09ADE00936400A4
:1004F00010936500089513DE44DE30E2E7DD0895D1
:100500007727D0E0CFE641E4342F59DF02F902FD2E
:100510001AC060E458E0342F10EF5EDF11274FD08F
:100520004ED0133081F0113011F411271CC012305D
:1005300011F410E818C0361711F410E814C038F0A0
:1005400010E0462F10C070936E0001E00895C8506F
:10055000188108E0C00F052F0A95111F0A95E9F7C9
:10056000107809F4462F18D08695812B6A955A95F4
:10057000A9F6899358E08827603081F67395431770
:1005800021F470936E0000E00895763009F0BDCF3D
:1005900070936E0002E00895C298BA9A00000000BD
:1005A000000000000000111F10F4C29ABA981795BD
:1005B000ADE071DEC29ABA98A1E06DDE0895C298EE
:1005C000BA9AA1E068DEC29ABA98A1E064DE110F7F
:1005D000B2991160ADE05FDE0895F1DE02F902FD2F
:1005E00003C08EDF002341F035E670DD32E76EDDBB
:1005F00032E76CDD30E222C030916E003063ACDE59
:1006000065DDAADE40DFDBDE21DF00916E00D0E099
:10061000CFE60F93DF93CF9353DF5CDFE2EBF3E0A2
:10062000009164001091650066DF96DECF91DF9146
:1006300008E0C00F0F910A9561F761CE8DDE46DDAF
:100640008BDEEAE4F6E06BDD5ACE2A2A48414C54B0
:100650002A2A0D0A0A0080DE8DD0F89400E20BBF32
:1006600008E005BB789430E030936100F894A7DE91
:10067000789402F902FD35C0F89442DF78940023A3
:1006800081F5F8949CDEE2DE789400916E00D0E073
:10069000CFE60F93DF93CF9313DF1CDF009164004D
:1006A0001091650029DF42D0CF91DF9108E0C00FA3
:1006B0000F910A9571F750DE00916100002339F027
:1006C000409160004B31D9F030E03093610053DE4F
:1006D00000E205BF78948895F89400E005BFC6CF86
:1006E0001895EAEEF6E01BDDE7CF3E7061732064FB
:1006F00065206361707465757220210D0A003EDE0D
:10070000F89400E00BBFFBCD27DE20E030E0E2DD17
:10071000002351F0002F10E0000F111F000F111FD8
:1007200030DD15DE2395F3CF17DEE9CD2091620091
:10073000309163001695079516950795002FBEDD3D
:10074000239500E0BBDDC2E6D0E0299339930895FC
:10075000209100003091000000E0B0DDE4E6F7E019
:10076000DEDCCDCD454550524F4D20766964652085
:10077000210D0A0020E030E0ADDD002311F02395CB
:10078000FBCFC2E6D0E0299339930895E5DDB7CDDC
:10079000902FE2DD24DD372F99DC362F97DCDCDD6E
:0407A00031E44CCF25
:00000001FF
